:10000000A82803013B208316C03086058312861280
:1000100032302220203022201C302220362028306E
:100020002220063022200C302220080020302428F4
:100030009300130E1C2013080F39093C031CF93ED2
:10004000393C24289201252812169100110E2920EE
:1000500011080F391204860086162F208612DC3014
:100060009000900B31280800C03039280130392821
:10007000023022200F308F00900B3C288F0B3C2841
:1000800008008316DF3081008312970108000B1DE2
:1000900008000B1180308102950F950A9503050821
:1000A00014069406013903190800150896009501F5
:1000B00008309607160EFF3A0F3982076E286E2811
:1000C0006E286E286E286E286E286E289428732855
:1000D0007A207A207A207A2078286E289719971427
:1000E0009711171208007A207A207A207A207A282D
:1000F00003107B280314990C190D013003189C067A
:1001000003109B0C9C0C031C892808309C0684302F
:100110009B06171E08009A0B08001908971517145C
:10012000980008309A00080008309A00971DA2280D
:1001300078301B06031D97145C301C06031D9714B2
:10014000971C1715FF309B009C009711171608008D
:100150000120412038205030242065302420653093
:1001600024206B3024205030242061302420633040
:1001700024206B302420C42047201718C82097184B
:10018000D9201719DC20BC281D3084004014080039
:100190001710401CD1281818401004082B3A0319D6
:1001A000080018088000840A0408403A03198403F0
:1001B00008009710C4200800171184038403040862
:1001C000C000362024308400F0203E3024201D3032
:1001D0008400F02034202D3084000721C420080042
:1001E00006308C000310000C203A0319F928203A3D
:1001F0002420840A8C0BF228000C0F390319080004
:100200002D302420000C0F39303E1C200800103007
:100210008C0000088E0020300E02031C11290E08ED
:100220002420840A04084006031908008C0B0929BD
:10023000080004084006031D19291D308400080029
:02400E00F23F7F
:00000001FF
